:020000040000fa
:080000005c0504000000000093
:020000040000fa
:020000040002f8
:04afe000dfff00008f
:020000040000fa
:020000040002f8
:04afe400ffff00006b
:020000040000fa
:020000040002f8
:04afe80078ff0000ee
:020000040000fa
:020000040002f8
:04afec007dff0000e5
:020000040000fa
:020000040002f8
:04aff00078ff0000e6
:020000040000fa
:1000080000000000000000000000000000000000e8
:10001800540500000000000000000000000000007f
:100028000000000000000000000000002809000097
:100038000000000000000000000000006a09000045
:10004800ae0900000000000000000000620a000085
:10005800ce0a0000fa0a00000000000000000000bc
:100068000000000000000000000000000000000088
:100078000000000000000000000000000000000078
:10008800000000000000000000000000de09000081
:10009800200a00000000000000000000000000002e
:1000a8000000000000000000000000000000000048
:1000b8000000000000000000000000000000000038
:1000c8000000000000000000000000000000000028
:1000d8000000000000000000000000000000000018
:1000e8000000000000000000000000000000000008
:1000f80000000000000000000000000000000000f8
:1001080000000000000000000000000000000000e7
:1001180000000000000000000000000000000000d7
:10012800000000009a0a0000000000000000000023
:1001380000000000000000000000000000000000b7
:1001480000000000000000000000000000000000a7
:100158000000000000000000000000000000000097
:100168000000000000000000000000000000000087
:100178000000000000000000000000000000000077
:100188000000000000000000000000000000000067
:100198000000000000000000260b0000520b0000c9
:1001a8007e0b0000000000000000000000000000be
:1001b8000000000000000000000000000000000037
:1001c8000000000000000000000000000000000027
:1001d8000000000000000000000000000000000017
:1001e8000000000000000000000000000000000007
:1001f80000000000000000000000000000000000f7
:1002080000000000000000000000000000000000e6
:1002180000000000000000000000000000000000d6
:1002280000000000000000000000000000000000c6
:1002380000000000000000000000000000000000b6
:1002480000000000000000000000000000000000a6
:100258000000000000000000000000000000000096
:100268000000000000000000000000000000000086
:0c0278000000000000000000000000007a
:020000040000fa
:10040000d9d1bf00d851b7004220af00d871ec005d
:10041000d9d1d600d9d1b60000c0d200d9d1bf0001
:1004200000c0fd00d9f1b700d8d1bf0000c0fd0069
:100430000040d200d9d1b600d9d1bf0000c0fd0024
:10044000d9f1b7001040b200d8f1d600d8f1b6000b
:10045000d9f1d600c08e800000000600803e20004a
:10046000030007008100e900fcff3a0000000600dd
:10047000831f7800c20320000400bc006601510005
:10048000e0815900f23fb1000380b1000600350061
:10049000ee03090000000000423fb1000380b100fc
:1004a000fbff3d001200b000223fb000020035000b
:1004b0000280090000000000cf0178000000060063
:1004c0000001780010012000f04fb00004a0d60019
:1004d000fdff390000000600040020000300370083
:1004e000140020000100370014002000889fbe0087
:1004f0008a9fbe00841f7800170107004f00780014
:1005000011003300f0ff2f00838f6c0006003b00ca
:10051000040565000a00a7000800370009f0a600de
:100520001000200008003700820f5400838f5c0009
:10053000030039001000200001003e0000002000f0
:1005400009f0a7000000ea004f05be004f04be00fe
:100550000000e000000006000002be00e00f5000b6
:10056000e08f580002003500ce00070000000600b2
:100570000401be0061006100010020008301d10080
:100580000281d3000200700083807000c500070064
:100590000001be000100370003f0a200869fbe00ec
:1005a000889fbe008a9fbe008c9fbe00ea000700a5
:1005b0002c0133006450e1004f0032006420e10060
:1005c0005200320003826c0007003b000905d00096
:1005d0000306d000820f54000c065d0002003900b3
:1005e00002003200890178000306780085825500f8
:1005f00004003d000003fd008103fd008502ea00c8
:100600008b854200840f720002003b0060001000e6
:10061000e08018006011b8000005eb007a28e100c6
:100620000a00390006007800c75ddd00f707b20058
:10063000878075002d003700828171000a017800e3
:10064000610560008180d1000080d3008502e9004f
:10065000f9ff3b00060440008784480002003b008d
:1006600060041400e0841c000988a3000700320025
:100670008a81710082817100610164008904d10066
:100680000884d3008b05e800170037000978a30021
:1006900013003a000b00e000130034008b05e90062
:1006a0000804440089844c000a4474000978a300bb
:1006b0000d003a000b00e000070034008b05e90054
:1006c0000804440089844c0001003a000b0020001b
:1006d0000978a300f7ff32000001eb0002003700a9
:1006e000828171000a017800b80007000cf0a700b1
:1006f00001f0a000e40037006420e10002003a00ad
:10070000838f6c00e50033000801be000200be00cc
:10071000dd003700869fbe00889fbe008a9fbe0016
:100720008c9fbe008c000700ce00330003866c0057
:100730006450e1002e0032006420e10033003200fa
:100740006150e1002f0032006120e10031003200f1
:1007500085855500eb07b000090020000804200043
:10076000050037000804440089844c000a00310069
:100770000603430087834b000001530081815b0027
:10078000f8ff33000203be000800a0000804440084
:1007900089844c00f6ff3900c639dd0083017300ff
:1007a00001003200130020008904d1000884d30026
:1007b0000998a300050032000800a7000300a0006c
:1007c0008904d1000884d3008b05e8008904d10096
:1007d0000884d3000001eb000281d2007b000700f7
:1007e00001f0a1000cf0a70001f0a000a600370066
:1007f0006420e100a90032000801be000200be0032
:10080000f7ff37006120e100a40032006000b8006b
:10081000f3ff37000000200001f82700f0ff370049
:10082000829fbe000001be00530007000470a700b5
:1008300003f0a10003f8a30015003a006509b10018
:10084000110032000a0035006928e100030035007c
:10085000010028004f01be0000000500000040001c
:10086000818048008502e900fcff3a00060037005d
:10087000f88f4200060035008100d1000080d300cf
:100880008502e800fcff3a004f01be0000000600b0
:100890008000eb004f01be00000005000080fb005f
:1008a0008000eb00829fbe00889fbe008a9fbe0032
:1008b000010578000100e0000400350008003c005c
:1008c0000000e0002000320005003700600010004a
:1008d000e080180002003b0001f024001a003700fd
:1008e0000004be006011b8006b0920000982cf002f
:1008f000020039000882cf000441b0006942520072
:100900000e00320008003b0082817100610164002a
:100910008904d1000884d3008b05e8000442e80074
:10092000f9ff3a00050037000804440089844c00b0
:100930008b05e9000442e900fbff3a0023000700b1
:100940000af0a70001f0a0004f05be004f04be0052
:100950004f01be00000006000004be0006000700b4
:100960000003be000405be000200be000200070036
:10097000844f750000000600c70ade00f107b200d0
:10098000f50fb20008003200e1cf42000200320051
:100990000170a00024000500810f700001003200ea
:1009a0000408050044000500810f700002003a00b1
:1009b000140005008502e9000000400081c04800e5
:1009c000fcff3b000170a000240005008100200016
:1009d000618055000b003d000b00200061fe2f00e0
:1009e0000100e1001d00340082817100610164009a
:1009f0008904d1000884d3000000e800faff3a001f
:100a000071002000610064000300700002006000bb
:100a10000900320061044400e0844c000988a5000c
:100a2000050032008b05e8006808e10002003a008a
:100a30008904d1000884d300f20f20000258e1009d
:100a400005003d00c75ddd00f907b2008980750033
:100a500008007800000006000bf827008b007800e3
:100a6000000005000200be006450e10005003600f1
:100a70006420e100020036000968a30001003a008a
:100a80000800be000160a0004f06be004f05be007a
:100a90004f04be004f03be0000000600f0ff2f0011
:100aa000f1ff2700f8ff37000020ef000220ef00e1
:100ab000c088a900004006000f002100401d210051
:100ac00000018800000000000000eb000007780033
:100ad0000c000900002f78000007eb005420ef0005
:100ae0000e2eef001e2eef000000eb00411d210036
:100af0002b1e09008018780010aea90014aea800c3
:100b000040a7a900a100200054fe0700e002200039
:100b1000303a880044e7a90044c7a9004407a90067
:100b20004427a9004447a9004467a9004487a900b5
:100b3000300020000600fc003174200082072000f5
:100b4000a309200082487800834878008048780014
:100b5000113a8000618070000600fc0021742000c2
:100b600062042000730520008248780083487800e2
:100b7000804878004427ef00e0022000303a8800e7
:100b8000300020000d00fc0031742000820720009e
:100b9000a3092000824878008348780080487800c4
:100ba0000000200021742000620420007305200052
:100bb00082487800834878008048780042a7ae00d9
:100bc000feff3700813e200024fe070010c0b30066
:100bd00086e6b70090c2b300c4e6b700000220006a
:100be00000708800007025008070880010aea90099
:100bf000008ea900108ea900000ea900002ea900e9
:100c0000100ea900102ea90010aea90014aea80065
:100c1000008ea900048ea9004188a80041a8a9005f
:100c200041c8a8000021ef0002a1ef0004a1a80024
:100c30000481a9000068a9002068a80005e1a900b6
:100c400011a1a9001061a9001021a90010a1a800fc
:100c50001081a8000621ef00003320006008880002
:100c600000e8a9004388a90043a8a80043c8a80039
:100c700020e8a80011e1a90013a1a9001221a900f0
:100c800012a1a8001281a8004408a8004428a900c5
:100c90004448a9000a21ef000ea1ef000108a900b5
:100ca0002108a80013e1a8001fa1a9001ec1a900e6
:100cb0001ea1a8001e81a9001e61a9001e21a90075
:100cc0001421ef001aa1ef004d88a9004da8a9003a
:100cd0004dc8a8000368a9002368a8001fe1a90067
:100ce00021a1a90020c1a90020a1a8002081a9005c
:100cf0002021a9001821ef001ca1ef004e08a80038
:100d00004e28a8004e48a9000388a9002388a800ff
:100d100021e1a9002002a9002022a9002042a90067
:100d200020a2a9002062a9002082a90020e2a90037
:100d30002102a9002122a90070072000401188008b
:100d400022a2a90022c2a90022e2a90021e2a80051
:100d50002182a9004588a90045a8a80045c8a90086
:100d60002168a8002828a8002bc8a9002be8a90002
:100d70002c08a9000bc8a9000be8a9000c08a900c1
:100d800001eca90001aca900016ca900014ca9006b
:100d9000012ca900010ca90000eca900008ca900fd
:100da00000aca90000cca900000ca900002ca900ef
:100db000004ca900006ca900202cef00402cef0093
:100dc000602cef0004acef00020ca900022ca9007b
:100dd000024ca900262cef00462cef00662cef00f9
:100de000282cef00482cef00682cef000aacef0035
:100df00023eca80023cca90043eca80043cca90015
:100e000063eca80063cca900dabc2a001b322400e2
:100e100030002c00fa608800fb60880020618800a8
:100e2000dabc2a001b32240000002800fa60880087
:100e3000fb60880010618800dabc2a001b322400a5
:100e400030002c00fa608800fb6088002062880077
:100e5000dabc2a001b32240000002800fa60880057
:100e6000fb60880010628800dabc2a001b32240074
:100e700030002c00fa608800fb6088002063880046
:100e8000dabc2a001b32240000002800fa60880027
:100e9000fb6088001063880011eea90011aea90064
:100ea000116ea900a70037003f0037000020200086
:100eb00000618800002020000062880000202000df
:100ec00000638800020ca900022ca800024ca800b4
:100ed00004acef0028acef0048acef0068acef00ca
:100ee000262cef00462cef00662cef000aacef003a
:100ef00023eca80023cca90043eca80043cca90014
:100f000063eca80063cca900dabc2a001b322400e1
:100f100030002c00fa608800fb60880020618800a7
:100f2000dabc2a001b32240000002800fa60880086
:100f3000fb60880010618800dabc2a001b322400a4
:100f400030002c00fa608800fb6088002062880076
:100f5000dabc2a001b32240000002800fa60880056
:100f6000fb60880010628800dabc2a001b32240073
:100f700030002c00fa608800fb6088002063880045
:100f8000dabc2a001b32240000002800fa60880026
:100f9000fb6088001063880011eea90011aea90063
:100fa000116ea900670037003500370000102000df
:100fb00000618800001020000062880000102000fe
:100fc00000638800020ca900022ca800024ca800b3
:100fd0000a2cef0004acef00282cef005055250040
:100fe00040628800a0aa2a0040638800dabc2a0078
:100ff0001b32240030002c00fa608800fb6088005f
:1010000020618800dabc2a001b32240000002c007a
:10101000fa608800fb60880010618800dabc2a0052
:101020001b32240030002c00fa608800fb6088002e
:1010300020628800dabc2a001b32240000002c0049
:10104000fa608800fb60880010628800dabc2a0021
:101050001b32240030002c00fa608800fb608800fe
:1010600020638800dabc2a001b32240000002c0018
:10107000fa608800fb608800106388003100370048
:1010800030003700001020000061880000102000b0
:1010900000628800020ca900022ca800024ca800e3
:1010a0000a2cef0004acef00282cef000000240015
:1010b00040628800dabc2a001b32240030002c0079
:1010c000fa608800fb60880020618800dabc2a0092
:1010d0001b32240000002c00fa608800fb608800ae
:1010e00010618800dabc2a001b32240030002c007a
:1010f000fa608800fb60880020628800dabc2a0061
:101100001b32240000002c00fa608800fb6088007d
:1011100010628800dabc2a001b32240030002c0048
:10112000fa608800fb60880020638800dabc2a002f
:101130001b32240000002c00fa608800fb6088004d
:1011400010638800218ca900418ca900618ca90042
:10115000216ca900416ca900616ca900214ca90077
:10116000414ca900614ca90020eca80040eca8006b
:1011700060eca8003e2cef005e2cef007e2cef0010
:1011800001eca8000000eb00a1552100ff000900c0
:10119000805878003f72ef004072ef00da090700d4
:1011a000d90a070000332000308f880010c0b30038
:1011b000e8f1b70010c0b300e9f1b700e851e20070
:1011c00002003a00a50b070017003700e8d1bf0066
:1011d00080407800e1cf500002003a00b00c0700d8
:1011e00011003700e8d1bf0080407800e2cf500006
:1011f00002003a00bb0d07000b003700e8d1bf002a
:1012000080407800e3cf500002003a00c60e07008d
:1012100005003700e8d1bf0080407800e4cf5000df
:1012200001003a00d10f07004209070010cea900c3
:1012300014cea900fe31ef000032ef000232ef00c1
:101240000432ef000632ef000832ef004e013700a3
:10125000ff3ffc004200f8003600f8004400f800b0
:101260008e1f78000e0020000d000900be1f7800c0
:101270003200f8000100fc000068a9000021ef0026
:1012800013eeaf0004003700508f80001008880074
:1012900015eea80004003700c08f8000ec11b500e7
:1012a0001008880015eea900ff3ffc003200f9008d
:1012b000ae0120000d0009004f1778004f0778009d
:1012c0004400f9003600f9004200f9000100fc007a
:1012d00000400600ff3ffc004200f8003600f80026
:1012e0004400f8008e1f78000e0020000d00090059
:1012f000be1f78003200f8000100fc0000e8a900e1
:101300000621ef00308f8000600888000a52e2005a
:1013100001003600fe31ec000b52e2000100360005
:101320000232ec000c52e200010036000632ec0002
:10133000ff3ffc003200f900ae0120000d00090063
:101340004f1778004f0778004400f9003600f90085
:101350004200f9000100fc0000400600ff3ffc00d5
:101360004200f8003600f8004400f8008e1f7800b4
:101370000e0020000d000900be1f78003200f800aa
:101380000100fc000108a900128eaa00108ea9001d
:10139000ff3ffc003200f900ae0120000d00090003
:1013a0004f1778004f0778004400f9003600f90025
:1013b0004200f9000100fc0000400600ff3ffc0075
:1013c0004200f8003600f8004400f8008e1f780054
:1013d0000e0020000d000900be1f78003200f8004a
:1013e0000100fc000368a9001421ef0013aeaf0058
:1013f00004003700708f8000d008880015aea80068
:1014000004003700c08f8000f011b500d0088800bc
:1014100015aea900ff3ffc003200f900ae0120002c
:101420000d0009004f1778004f0778004400f900bd
:101430003600f9004200f9000100fc0000400600ff
:10144000ff3ffc004200f8003600f8004400f800be
:101450008e1f78000e0020000d000900be1f7800ce
:101460003200f8000100fc000388a9001821ef00f9
:10147000136eaf0004003700908f8000e0088800f2
:10148000156ea80004003700c08f8000f411b5006d
:10149000e0088800156ea900ff3ffc003200f9004b
:1014a000ae0120000d0009004f1778004f077800ab
:1014b0004400f9003600f9004200f9000100fc0088
:1014c00000400600ff3ffc004200f8003600f80034
:1014d0004400f8008e1f78000e0020000d00090067
:1014e000be1f78003200f8000100fc000168a9006e
:1014f0003f72ec003fd2bf008080fb0030118000c3
:10150000a255210080707900ff3ffc003200f900f5
:10151000ae0120000d0009004f1778004f0778003a
:101520004400f9003600f9004200f9000100fc0017
:1015300000400600ff3ffc004200f8003600f800c3
:101540004400f8008e1f78000e0020000d000900f6
:10155000be1f78003200f8000100fc000828a90036
:101560002242ae00000037002222af002222a90052
:10157000ff3ffc003200f900ae0120000d00090021
:101580004f1778004f0778004400f9003600f90043
:101590004200f9000100fc0000400600ff3ffc0093
:1015a0004200f8003600f8004400f8008e1f780072
:1015b0000e0020000d000900be1f78003200f80068
:1015c0000100fc000188a900ff3ffc003200f90087
:1015d000ae0120000d0009004f1778004f0778007a
:1015e0004400f9003600f9004200f9000100fc0057
:1015f00000400600ff3ffc004200f8003600f80003
:101600004400f8008e1f78000e0020000d00090035
:10161000be1f78003200f8000100fc0001a8a900fc
:10162000ff3ffc003200f900ae0120000d00090070
:101630004f1778004f0778004400f9003600f90092
:101640004200f9000100fc0000400600ff3ffc00e2
:101650004200f8003600f8004400f8008e1f7800c1
:101660000e0020000d000900be1f78003200f800b7
:101670000100fc000bc8a900ff3ffc003200f9008c
:10168000ae0120000d0009004f1778004f077800c9
:101690004400f9003600f9004200f9000100fc00a6
:1016a00000400600ff3ffc004200f8003600f80052
:1016b0004400f8008e1f78000e0020000d00090085
:1016c000be1f78003200f8000100fc000be8a90002
:1016d000ff3ffc003200f900ae0120000d000900c0
:1016e0004f1778004f0778004400f9003600f900e2
:1016f0004200f9000100fc0000400600ff3ffc0032
:101700004200f8003600f8004400f8008e1f780010
:101710000e0020000d000900be1f78003200f80006
:101720000100fc000c08a900ff3ffc003200f9009a
:10173000ae0120000d0009004f1778004f07780018
:101740004400f9003600f9004200f9000100fc00f5
:101750000040060040d2bf003f52e30007003200c5
:101760004072ec0040d2bf000080fb00a155210078
:1017700060c0780041f2b7000100370041f2ef008d
:101780000000060000000600f2ff070090cdb30045
:101790004152b50006003900e0cfb3004152b50018
:1017a00001003900010037004272ef000f033700db
:1017b00041f2ae002f0037004272ef0080c8b30044
:1017c0004152e30005003a0041d2bf0042f2b700a7
:1017d00043f2ef0044f2ef002500370080c9b30068
:1017e0004152e30005003a0041d2bf0042f2b70087
:1017f00045f2ef0046f2ef001d00370080cab3004b
:101800004152e30005003a0041d2bf0042f2b70066
:1018100047f2ef0048f2ef001500370080cbb3002d
:101820004152e30005003a0041d2bf0042f2b70046
:1018300049f2ef004af2ef000d00370080ccb30010
:101840004152e30004003a0041d2bf0042f2b70027
:101850004bf2ef000600370080cdb3004152e300a9
:1018600003003a0041d2bf0042f2b7004cf2ef0051
:10187000de0237004252e20002003a00db0237008b
:10188000da02370080c8b3004252e30069003a0030
:1018900000e0ef004352e30003003a0041d2bf00f2
:1018a00043f2b700620037004152ec0044f2b70047
:1018b000c200200043d2bf000080fb000200e00015
:1018c00002003200110009000280d800a18e8800b9
:1018d000d631ef00a08e8000b18e8000e70f50005f
:1018e000e08f580018003a0040c0b3000af2b70079
:1018f000fbd1bf00e9fb0700709088008190880051
:1019000044d2bf00e5fb07000001be0070908000dc
:10191000819080007ffb0700d0908800e1908800d4
:10192000fbd1bf000080fb0000004000a14521006a
:101930006080780030618800fe31ef000032ef00f7
:1019400011e1a80039003700a08e8000b18e800020
:10195000e80f5000e08f580018003a0040c0b30074
:101960000bf2b700fcd1bf00ccfb0700f090880061
:101970000191880044d2bf00c8fb07000001be00ef
:10198000f09080000191800062fb07005091880078
:1019900061918800fcd1bf000080fb000000400086
:1019a000a145210060807800306288000232ef009b
:1019b0000432ef0011e1a8001c003700a08e800067
:1019c000b18e8000e90f5000e08f580017003a00f8
:1019d00040c0b3000cf2b700fdd1bf00affb070061
:1019e000709188008191880044d2bf00abfb070052
:1019f0000001be00709180008191800045fb0700ce
:101a0000d0918800e1918800fdd1bf000080fb00eb
:101a100000004000a145210060807800306388000c
:101a20000632ef000832ef0011e1a80043f2ef00a8
:101a30006e02370080c9b3004252e30031023a001f
:101a400000e0ef004552e30003003a0041d2bf003e
:101a500045f2b7002a02370041d2bf0046f2b70074
:101a60004652e20060003a00c200200045d2bf00aa
:101a70000080fb000200e0000200320011000900bb
:101a80000280d800a18e8800d631ef00a08e8000a1
:101a9000b18e8000e70f5000e08f580018003a0028
:101aa00040c0b3000af2b700fbd1bf007bfb0700c8
:101ab000709088008190880058d2bf0077fb0700a3
:101ac0000001be00709080008190800011fb070033
:101ad000d0908800e1908800fbd1bf000080fb001f
:101ae00000004000a145210060807800306188003e
:101af000fe31ef000032ef0011e1a800390037009d
:101b0000a08e8000b18e8000e80f5000e08f58005a
:101b100018003a0040c0b3000bf2b700fcd1bf0080
:101b20005efb0700f09088000191880058d2bf004a
:101b30005afb07000001be00f09080000191800078
:101b4000f4fa07005091880061918800fcd1bf0031
:101b50000080fb0000004000a1452100608078006b
:101b6000306288000232ef000432ef0011e1a80079
:101b70001c003700a08e8000b18e8000e90f50005d
:101b8000e08f580017003a0040c0b3000cf2b700d5
:101b9000fdd1bf0041fb0700709188008191880052
:101ba00058d2bf003dfb07000001be0070918000cd
:101bb00081918000d7fa0700d0918800e1918800d8
:101bc000fdd1bf000080fb0000004000a1452100c6
:101bd00060807800306388000632ef000832ef0042
:101be00011e1a800c601370045d2bf00804078004f
:101bf000ffcf500023003a0045d2bf0050f2b7009b
:101c000046d2bf000080fb00f08e880010c0b300f9
:101c10000af2b7000e32ef001032ef00262cef0070
:101c200056d2bf001dfb07000001be00f08e8000f1
:101c30001bfb0700b7fa070090908800a19088006e
:101c4000fe31ef000032ef0011e1a80053d2bf00d7
:101c50000080fb00520920000200b800508f88006d
:101c6000508f8000a157290000805000608f8800ad
:101c700015eea9000068a9002068a80005e1a800e9
:101c80009e01370000c2b3004552e30023003a0032
:101c900045d2bf0051f2b70046d2bf000080fb0022
:101ca000008f880010c0b3000bf2b7001e32ef00a7
:101cb0002032ef00462cef0056d2bf00f7fa0700a3
:101cc0000001be00008f8000f5fa070091fa0700be
:101cd00010918800219188000232ef000432ef0059
:101ce00011e1a80054d2bf000080fb00d208200000
:101cf0000200b800708f8800708f800061d12800ca
:101d000000805000808f880015aea9000368a900ec
:101d10002368a8001fe1a8007801370010c2b300b3
:101d20004552e30023003a0045d2bf0052f2b7000b
:101d300046d2bf000080fb00108f880010c0b300a7
:101d40000cf2b7002e32ef003032ef00662cef00bd
:101d500056d2bf00d1fa07000001be00108f8000ec
:101d6000cffa07006bfa070090918800a1918800d4
:101d70000632ef000832ef0011e1a80055d2bf0093
:101d80000080fb00520820000200b800908f8800fd
:101d9000908f8000b152280000805000a08f8800f2
:101da000156ea9000388a9002388a80021e1a800d6
:101db00052013700b0c2b3004552e30023003a009d
:101dc00045d2bf0050f2b70046d2bf000080fb00f2
:101dd000f08e880010c0b3000af2b7000e32ef0098
:101de0001032ef00262cef0056d2bf00abfa0700ee
:101df0000001be00f08e8000a9fa070045fa070036
:101e000090908800a1908800fe31ef000032ef0032
:101e100011e1a80053d2bf000080fb00a204200003
:101e20000200b800508f8800508f8000d1ab240092
:101e300000805000608f880015eea9000068a9009e
:101e40002068a80005e1a8002c013700c0c2b3003b
:101e50004552e30023003a0045d2bf0051f2b700db
:101e600046d2bf000080fb00008f880010c0b30086
:101e70000bf2b7001e32ef002032ef00462cef00cd
:101e800056d2bf0085fa07000001be00008f800017
:101e900083fa07001ffa070010918800219188003b
:101ea0000232ef000432ef0011e1a80054d2bf006b
:101eb0000080fb00620420000200b800708f8800e0
:101ec000708f8000b168240000805000808f8800ef
:101ed00015aea9000368a9002368a8001fe1a800a7
:101ee00006013700d0c2b3004552e30023003a0098
:101ef00045d2bf0052f2b70046d2bf000080fb00bf
:101f0000108f880010c0b3000cf2b7002e32ef0023
:101f10003032ef00662cef0056d2bf005ffa0700a8
:101f20000001be00108f80005dfa0700f9f907007c
:101f300090918800a19188000632ef000832ef00ee
:101f400011e1a80055d2bf000080fb002204200050
:101f50000200b800908f8800908f800051292400e3
:101f600000805000a08f8800156ea9000388a9008a
:101f70002388a80021e1a800e000370070c3b30067
:101f80004552e30023003a0045d2bf0050f2b700ab
:101f900046d2bf000080fb00f08e880010c0b30066
:101fa0000af2b7000e32ef001032ef00262cef00dd
:101fb00056d2bf0039fa07000001be00f08e800043
:101fc00037fa0700d3f9070090908800a1908800a5
:101fd000fe31ef000032ef0011e1a80053d2bf0044
:101fe0000080fb00520220000200b800508f8800e1
:101ff000508f8000e155220000805000608f8800e3
:1020000015eea9000068a9002068a80005e1a80055
:10201000ba00370080c3b3004552e30023003a0002
:1020200045d2bf0051f2b70046d2bf000080fb008e
:10203000008f880010c0b3000bf2b7001e32ef0013
:102040002032ef00462cef0056d2bf0013fa0700f3
:102050000001be00008f800011fa0700adf90700f3
:1020600010918800219188000232ef000432ef00c5
:1020700011e1a80054d2bf000080fb003202200012
:102080000200b800708f8800708f800051342200e9
:1020900000805000808f880015aea9000368a90059
:1020a0002368a8001fe1a8009400370090c3b30084
:1020b0004552e30023003a0045d2bf0052f2b70078
:1020c00046d2bf000080fb00108f880010c0b30014
:1020d0000cf2b7002e32ef003032ef00662cef002a
:1020e00056d2bf00edf907000001be00108f80003e
:1020f000ebf9070087f9070090918800a19188000b
:102100000632ef000832ef0011e1a80055d2bf00ff
:102110000080fb00120220000200b800908f8800af
:10212000908f8000a114220000805000a08f8800b2
:10213000156ea9000388a9002388a80021e1a80042
:102140006e00370030c4b3004552e30022003a006d
:1021500045d2bf0050f2b70046d2bf000080fb005e
:10216000f08e880010c0b3000af2b7000e32ef0004
:102170001032ef00262cef0056d2bf00c7f907003f
:102180000001be00f08e8000c5f9070061f907006c
:1021900090908800a1908800fe31ef000032ef009f
:1021a00011e1a80053d2bf000080fb007200b8000c
:1021b000508f8800508f8000f12a2100008050004d
:1021c000608f880015eea9000068a9002068a800ab
:1021d00005e1a8004900370040c4b3004552e300c0
:1021e00022003a0045d2bf0051f2b70046d2bf00ec
:1021f0000080fb00008f880010c0b3000bf2b70016
:102200001e32ef002032ef00462cef0056d2bf0006
:10221000a2f907000001be00008f8000a0f90700ae
:102220003cf9070010918800219188000232ef00ec
:102230000432ef0011e1a80054d2bf000080fb007f
:102240007100b800708f8800708f8000211a210003
:1022500000805000808f880015aea9000368a90097
:102260002368a8001fe1a8002400370050c4b30071
:102270004552e30021003a0045d2bf0052f2b700b8
:1022800046d2bf000080fb00108f880010c0b30052
:102290000cf2b7002e32ef003032ef00662cef0068
:1022a00056d2bf007df907000001be00108f8000ec
:1022b0007bf9070017f9070090918800a191880029
:1022c0000632ef000832ef0011e1a80055d2bf003e
:1022d0000080fb007000b800908f8800908f800015
:1022e000510a210000805000a08f8800156ea900bf
:1022f0000388a9002388a80021e1a80045f2ef0087
:102300003a00370080cab3004252e3000a003a00a4
:1023100000e0ef004752e30003003a0041d2bf0063
:1023200047f2b7000300370041d2bf0048f2b700c0
:10233000d10207002d00370080cbb3004252e300ea
:102340000a003a0000e0ef004952e30003003a00bf
:1023500041d2bf0049f2b7000300370041d2bf00ad
:102360004af2b700c30307002000370080ccb30057
:102370004252e30007003a0000e0ef004b52e30056
:1023800003003a0041d2bf004bf2b7006d030700d3
:102390001600370080cdb3004252e30007003a0038
:1023a00000e0ef004c52e30003003a0041d2bf00ce
:1023b0004cf2b700950307000c00370080ceb30045
:1023c0004252e30009003a0000e0ef004d52e30002
:1023d00003003a0041d2bf004df2b70003003700be
:1023e00041d2bf004ef2b700850307005090800035
:1023f00061908000e00f5000e08f58000a003a0022
:1024000011e1ae000700370011e1a900fe31ef0035
:102410000032ef000232ef000432ef000632ef002c
:102420000832ef00880237000a52e20002003a0048
:10243000d5003700d40037000ad2bf0080407800b2
:10244000e1cf500055003a0001908000f08f8000ed
:10245000808f5000500031000032ec00f08e800080
:102460000ff907000001be0070908000819080008d
:102470001df8070048003d007290800083908000a6
:1024800090908000a190800044f807007090880030
:10249000819088007290800083908000f08e800090
:1024a000fff8070010f8070031003d00f08e8000b3
:1024b000fbf807007090880081908800f28e800001
:1024c00002014100a04521006000790030618800d0
:1024d000fad1bf000081fb0003002000f08e8000d5
:1024e0000100200000015100818159000200be005e
:1024f00019f80700b0908800c190880057d2bf003b
:10250000e6f807000001be00b0908000c190800096
:1025100080f80700b0908800c19088006011b80072
:10252000b0908000c1908000ebf707000a003a00ed
:10253000fad1bf000080fb0000004000a14521004f
:1025400060807800306188000a72ef00fe31ef0091
:102550000032ef000500370020c0b3000af2b700d8
:10256000fe31ef000032ef0011e1a8000a00370051
:102570007090800081908000a9f807004ff2b700aa
:102580004fd2bf000080fb0000004000a1452100a9
:1025900060807800306188007b0037000ad2bf007d
:1025a00080407800e2cf50004d003a00019080005a
:1025b000f08f8000808f5000480031000032ec0026
:1025c0007290800083908000b0908000c190800065
:1025d000f2f70700709088008190880011f2ae0039
:1025e000020037000e32ef001032ef0019f2ae0099
:1025f0001c0037007290800083908000fad1bf00e9
:10260000a6f80700b8f707000c003d0070908000a6
:102610008190800082f807004ff2b7004fd2bf00d0
:102620000080fb0000004000a14521006080780090
:102630003061880011e1a80009003700fad1bf001d
:102640000080fb0000004000a14521006080780070
:10265000306188000a72ef00fe31ef000032ef00b7
:102660001e00370019f2af001c003700fad1bf007e
:102670008af807000001be00709080008190800001
:1026800099f707000c003d00709080008190800059
:1026900063f807004ff2b7004fd2bf000080fb0085
:1026a00000004000a1452100608078003061880072
:1026b00011e1a80009003700fad1bf000080fb003b
:1026c00000004000a1452100608078003061880052
:1026d0000a72ef00fe31ef000032ef002a003700ef
:1026e0000ad2bf0080407800e4cf500026003a00b4
:1026f00001908000f08f8000808f50002200310018
:102700000032ec007090800081908000d2908000b8
:10271000e3908000a0f70700709088008190880007
:102720000200200003002000709080008190800053
:102730006bf707000a003c000a72ef00262cef003e
:10274000fe31ef000032ef005072ef002068a90068
:102750000068a90005e1a90015eea9000a003700ec
:1027600070908000819080002df807004ff2b70034
:102770004fd2bf000080fb0000004000a1452100b7
:1027800060807800306188000b52e20002003a005d
:10279000d5003700d40037000bd2bf00804078004e
:1027a000e1cf500055003a00219080001090800049
:1027b000808f5000500031000432ec00008f800008
:1027c00037f807000001be00f09080000191800002
:1027d00043f7070048003c00f2908000039180001e
:1027e00010918000219180006cf70700f090880024
:1027f00001918800f290800003918000008f80009a
:1028000027f8070038f7070031003d00008f8000ef
:1028100023f80700f090880001918800028f800063
:1028200002014100a045210060007900306288006b
:10283000fad1bf000081fb0003002000008f800060
:102840000100200000015100818159000200be00fa
:1028500041f70700309188004191880057d2bf00ae
:102860000ef807000001be00309180004191800009
:10287000a8f7070030918800419188006011b800e6
:10288000309180004191800013f707000a003a0060
:10289000fad1bf000080fb0000004000a1452100ec
:1028a00060807800306288000b72ef000232ef0027
:1028b0000432ef000500370020c0b3000bf2b70070
:1028c0000232ef000432ef0011e1a8000a003700e5
:1028d000f090800001918000d1f707004ff2b7001f
:1028e0004fd2bf000080fb0000004000a145210046
:1028f00060807800306288007b0037000bd2bf0018
:1029000080407800e2cf50004d003a0021908000d6
:1029100010908000808f5000480031000432ec009d
:10292000f2908000039180003091800041918000fe
:102930001af70700f09088000191880021f2ae009c
:10294000020037001e32ef002032ef0029f2ae0005
:102950001c003700f290800003918000fad1bf0084
:10296000cef70700e0f607000c003d00f090800075
:1029700001918000aaf707004ff2b7004fd2bf00c5
:102980000080fb0000004000a1452100608078002d
:102990003062880011e1a80009003700fad1bf00b9
:1029a0000080fb0000004000a1452100608078000d
:1029b000306288000b72ef000232ef000432ef0049
:1029c0001e00370029f2af001c003700fad1bf000b
:1029d000b2f707000001be00f09080000191800076
:1029e000c1f607000c003d00f090800001918000ce
:1029f0008bf707004ff2b7004fd2bf000080fb00fb
:102a000000004000a145210060807800306288000d
:102a100011e1a80009003700fad1bf000080fb00d7
:102a200000004000a14521006080780030628800ed
:102a30000b72ef000232ef000432ef002a00370081
:102a40000bd2bf0080407800e4cf500026003a004f
:102a50002190800010908000808f50002200310073
:102a60000432ec00f09080000191800052918000cf
:102a700063918000c8f60700f090880001918800fb
:102a80000200200003002000f090800001918000ef
:102a900093f607000a003c000b72ef00462cef0093
:102aa0005172ef000232ef000432ef002368a900f8
:102ab0000368a9001fe1a90015aea9000a003700ac
:102ac000f09080000191800055f707004ff2b700a9
:102ad0004fd2bf000080fb0000004000a145210054
:102ae00060807800306288000c52e20002003a00f8
:102af000d5003700d40037000cd2bf0080407800ea
:102b0000e1cf500055003a004190800030908000a5
:102b1000808f5000500031000832ec00108f800090
:102b20005ff707000001be00709180008191800076
:102b30006bf6070048003c00729180008391800092
:102b400090918000a191800094f607007091880018
:102b5000819188007291800083918000108f8000a5
:102b60004ff7070060f6070031003d00108f80002e
:102b70004bf707007091880081918800128f8000c8
:102b800002014100a0452100600079003063880007
:102b9000fad1bf000081fb0003002000108f8000ed
:102ba0000100200000015100818159000200be0097
:102bb00069f60700b0918800c191880057d2bf0024
:102bc00036f707000001be00b0918000c19180007f
:102bd000d0f60700b0918800c19188006011b8005c
:102be000b0918000c19180003bf607000a003a00d6
:102bf000fad1bf000080fb0000004000a145210089
:102c000060807800306388000c72ef000632ef00bd
:102c10000832ef000500370020c0b3000cf2b70007
:102c20000632ef000832ef0011e1a8000a00370079
:102c30007091800081918000f9f607004ff2b70093
:102c40004fd2bf000080fb0000004000a1452100e2
:102c500060807800306388007b0037000cd2bf00b2
:102c600080407800e2cf50004d003a004190800053
:102c700030908000808f5000480031000832ec0016
:102c80007291800083918000b0918000c19180009a
:102c900042f60700709188008191880031f2ae0001
:102ca000020037002e32ef003032ef0039f2ae0072
:102cb0001c0037007291800083918000fad1bf0020
:102cc000f6f6070008f607000c003d007091800042
:102cd00081918000d2f607004ff2b7004fd2bf00bb
:102ce0000080fb0000004000a145210060807800ca
:102cf0003063880011e1a80009003700fad1bf0055
:102d00000080fb0000004000a145210060807800a9
:102d1000306388000c72ef000632ef000832ef00db
:102d20001e00370039f2af001c003700fad1bf0097
:102d3000daf607000001be007091800081918000ea
:102d4000e9f507000c003d00709180008191800042
:102d5000b3f607004ff2b7004fd2bf000080fb0070
:102d600000004000a14521006080780030638800a9
:102d700011e1a80009003700fad1bf000080fb0074
:102d800000004000a1452100608078003063880089
:102d90000c72ef000632ef000832ef002a00370015
:102da0000cd2bf0080407800e4cf500026003a00eb
:102db0004190800030908000808f500022003100d0
:102dc0000832ec007091800081918000d2918000e7
:102dd000e3918000f0f507007091880081918800f0
:102de000020020000300200070918000819180008b
:102df000bbf507000a003c000c72ef00662cef00e8
:102e00005272ef000632ef000832ef002388a9006b
:102e10000388a90021e1a900156ea9000a00370066
:102e200070918000819180007df607004ff2b7001d
:102e30004fd2bf000080fb0000004000a1452100f0
:102e400060807800306388006df50700a08e8800f0
:102e5000b08f8000d411b600e08e8800b08f800063
:102e6000d08e8800da31d500e08e8000da11b5000e
:102e7000c08f880044fa370047d2bf0080407800f6
:102e8000ffcf50000c003a004852ec0053f2b7005c
:102e900053d2bf000080fb00520920000200b8009e
:102ea000508f8800508f8000a1572900008050006b
:102eb000608f8800a100370000c2b3004752e300d2
:102ec0000c003a004852ec0054f2b70054d2bf0054
:102ed0000080fb00d20820000200b800708f88003c
:102ee000708f800061d1280000805000808f8800a2
:102ef0009200370010c2b3004752e3000c003a00c2
:102f00004852ec0055f2b70055d2bf000080fb00dc
:102f1000520820000200b800908f8800908f800037
:102f2000b152280000805000a08f88008300370035
:102f3000b0c2b3004752e3000c003a004852ec0024
:102f400053f2b70053d2bf000080fb00a204200060
:102f50000200b800508f8800508f8000d1ab240051
:102f600000805000608f880074003700c0c2b3003a
:102f70004752e3000c003a004852ec0054f2b7000c
:102f800054d2bf000080fb00620420000200b800a1
:102f9000708f8800708f8000b1682400008050001e
:102fa000808f880065003700d0c2b3004752e3002d
:102fb0000c003a004852ec0055f2b70055d2bf0061
:102fc0000080fb00220420000200b800908f8800df
:102fd000908f80005129240000805000a08f88002d
:102fe0005600370070c3b3004752e3000c003a00ac
:102ff0004852ec0053f2b70053d2bf000080fb00f0
:10300000520220000200b800508f8800508f8000cc
:10301000e155220000805000608f88004700370093
:1030200080c3b3004752e3000c003a004852ec0062
:1030300054f2b70054d2bf000080fb0032022000df
:103040000200b800708f8800708f80005134220019
:1030500000805000808f88003800370090c3b30094
:103060004752e3000c003a004852ec0055f2b7001a
:1030700055d2bf000080fb00120220000200b80001
:10308000908f8800908f8000a11422000080500053
:10309000a08f88002900370030c4b3004752e300f6
:1030a0000b003a004852ec0053f2b70053d2bf0075
:1030b0000080fb007200b800508f8800508f8000a5
:1030c000f12a210000805000608f88001b0037002b
:1030d00040c4b3004752e3000b003a004852ec00f2
:1030e00054f2b70054d2bf000080fb007100b8005a
:1030f000708f8800708f8000211a2100008050009e
:10310000808f88000d00370050c4b3004752e300a1
:103110000a003a004852ec0055f2b70055d2bf0001
:103120000080fb007000b800908f8800908f8000b6
:10313000510a210000805000a08f880047f2ef0064
:10314000000006004b52e20002003a00790107003d
:10315000290037004bd2bf0080407800e1cf5000fb
:1031600002003a0089010700230037004bd2bf005c
:1031700080407800e2cf500002003a009a01070038
:103180001d0037004bd2bf0080407800e3cf5000d5
:1031900002003a00ab010700170037004bd2bf0016
:1031a00080407800e4cf500002003a00bc010700e4
:1031b000110037004bd2bf0080407800e5cf5000af
:1031c00002003a00cd0107000b0037004bd2bf00d0
:1031d00080407800e6cf500002003a00c8010700a6
:1031e000050037004bd2bf0080407800e7cf500089
:1031f00001003a00c30107004bf2ef000000060097
:103200004df2ef004ef2ef00000006005052e200d7
:10321000060036004cd2bf000080fb0000004000da
:10322000a145210060807800306188005152e200a1
:10323000060036004cd2bf000080fb0000004000ba
:10324000a145210060807800306288005252e2007f
:10325000060036004cd2bf000080fb00000040009a
:10326000a145210060807800306388004cf2ef00b7
:103270000000060049d2bf0080407800e1cf500036
:1032800009003a004ad2bf000080fb004300dd0085
:10329000b08f88004ad2bf000080fb0088f407008e
:1032a00059f2b700e600370049d2bf0080407800ed
:1032b000e7cf500009003a004ad2bf00faf1b70048
:1032c000fad1bf00fbf1b700fad1bf00fcf1b700a3
:1032d000fad1bf00fdf1b700d900370049d2bf00d5
:1032e00080407800eecf500008003a004a72ec00af
:1032f0004ad2bf0053f2b7004ad2bf0054f2b7001f
:103300004ad2bf0055f2b700cd00370049d2bf0006
:1033100080407800efcf500009003a004ad2bf0049
:103320000080fb00208f8800e411ec004400dd00e9
:10333000308f880000072000e631b400c00037005d
:1033400049d2bf0080407800f0cf500003003a001f
:103350004a52ec0056f2b700b900370049d2bf001c
:1033600080407800f2cf500003003a004a52ec004f
:1033700057f2b700b200370049d2bf008040780052
:10338000f3cf500003003a004a52ec0058f2b70065
:10339000ab00370020c4b3004952e30008003a00f4
:1033a0004a52e20003003a00a700070014aea8004a
:1033b0000200370014aea900048ea800a000370058
:1033c00000c5b3004952e30027003a004a52ec001e
:1033d000e8f1b700e8d1bf000080fb004500de0047
:1033e000e8f1b700e9d1bf00e851e3001d00320069
:1033f000e851e20002003a00180307001700370006
:10340000e8d1bf0080407800e1cf500002003a00d0
:103410002304070011003700e8d1bf008040780086
:10342000e2cf500002003a002e0507000b003700e3
:10343000e8d1bf0080407800e3cf500002003a009e
:103440003906070005003700e8d1bf00804078004a
:10345000e4cf500001003a0044070700e8d1bf0064
:10346000e9f1b70076003700a0c5b3004952e30088
:1034700022003a005052e20007003600262cef00ee
:103480000a72ef002068a90015eea9005072ef0043
:10349000fe31ef000032ef005152e200070036002b
:1034a000462cef000b72ef002368a90015aea900af
:1034b0005172ef000232ef000432ef005252e2008c
:1034c00007003600662cef002388a9000c72ef007d
:1034d000156ea9005272ef000632ef000832ef00bd
:1034e0005090800061908000e00f5000e08f580005
:1034f00001003a0011e1a9005100370070c6b30085
:103500004952e30010003a005052e2000b0036002e
:103510000a52e20008003a004ad2bf000080fb00d5
:1035200000004000a14521006080780030618800e3
:103530004ad2bf00fbf1b70002003700fad1bf004a
:10354000fbf1b7003e00370080c6b3004952e300ec
:1035500010003a005152e2000b0036000b52e2001c
:1035600008003a004ad2bf000080fb000000400083
:10357000a145210060807800306288004ad2bf00f7
:10358000fcf1b70002003700fad1bf00fcf1b70030
:103590002b00370090c6b3004952e30010003a00f8
:1035a0005252e2000b0036000c52e20008003a00d2
:1035b0004ad2bf000080fb0000004000a14521006e
:1035c00060807800306388004ad2bf00fdf1b70008
:1035d00002003700fad1bf00fdf1b7001800370034
:1035e000b0c7b3004952e30015003a00262cef00a3
:1035f000462cef00662cef000a32ef000c32ef0091
:1036000011e1a9002068a9002368a9002388a90066
:1036100015eea90015aea900156ea9005072ef00b5
:103620005172ef005272ef00fe31ef000032ef00f6
:103630000232ef000432ef000632ef000832ef00f2
:1036400049f2ef0000000600262cef00462cef00a8
:10365000662cef0014aea800048ea9000a32ef0019
:103660000c32ef0011e1a9002068a9002368a9002d
:103670002388a90011eea90015eea90011aea9003a
:1036800015aea900116ea900156ea9005072ef00c9
:103690005172ef005272ef00fe31ef000032ef0086
:1036a0000232ef000432ef000632ef000832ef0082
:1036b00000342000308f88001e00070010c0b300c7
:1036c000e8f1b700e851e20002003a0063020700a7
:1036d00017003700e8d1bf0080407800e1cf5000ec
:1036e00002003a006e03070011003700e8d1bf0066
:1036f00080407800e2cf500002003a0079040700d1
:103700000b003700e8d1bf0080407800e3cf5000c5
:1037100002003a008405070005003700e8d1bf0029
:1037200080407800e4cf500001003a008f06070087
:103730000000060080c0b30056f2b70060c0b300be
:1037400057f2b70060c5b300faf1b700fad1bf0075
:10375000fbf1b700fad1bf00fcf1b700fad1bf000e
:10376000fdf1b700a0c0b30058f2b70000c8b30025
:1037700053f2b70000c8b30054f2b70000c8b3005a
:1037800055f2b700f631ef000000060020c0b3008c
:1037900056f2b70010c0b30057f2b700c0c1b30073
:1037a000faf1b700fad1bf00fbf1b700fad1bf00c0
:1037b000fcf1b700fad1bf00fdf1b700e0c1b300e2
:1037c00058f2b700b0c0b30053f2b700b0c0b300b6
:1037d00054f2b700b0c0b30055f2b7004006200065
:1037e000b08f88000000060090c1b30056f2b70009
:1037f000a0c0b30057f2b70080c7b300faf1b7001a
:10380000fad1bf00fbf1b700fad1bf00fcf1b7005d
:10381000fad1bf00fdf1b70020c3b30058f2b700e2
:1038200030c0b30053f2b70030c0b30054f2b70059
:1038300030c0b30055f2b70060092000b08f880097
:103840000000060080c0b30056f2b70020c0b300ed
:1038500057f2b70040c6b300faf1b700fad1bf0083
:10386000fbf1b700fad1bf00fcf1b700fad1bf00fd
:10387000fdf1b700a0c0b30058f2b70000c5b30017
:1038800053f2b70000c5b30054f2b70000c5b3004f
:1038900055f2b700a0002000b08f8800000006009d
:1038a00010c0b30056f2b70010c0b30057f2b70013
:1038b000f0c7b300faf1b700fad1bf00fbf1b700cf
:1038c000fad1bf00fcf1b700fad1bf00fdf1b7009b
:1038d00040c1b30058f2b70030c0b30053f2b70094
:1038e00030c0b30054f2b70030c0b30055f2b70097
:1038f000401f2000b08f8800000006000000060076
:1039000000000600000006005ab2ef00a0c7250024
:10391000e092880050982500f092880040812500b0
:1039200000938800906a2500109388003054250089
:1039300020938800303e2500309388009028250091
:1039400040938800501325005093880060fe2400a7
:1039500060938800c0e924007093880080d524001b
:103960008093880090c1240090938800f0ad2400db
:10397000a0938800a09a2400b0938800a087240018
:10398000c0938800f0742400d093880090622400d3
:10399000e093880080502400f0938800b03e24001b
:1039a00000948800302d240010948800f01b24001f
:1039b00020948800000b24003094880050fa2300e3
:1039c00040948800e0e9230050948800c0d9230087
:1039d00060948800e0c923007094880040ba2300f6
:1039e00080948800e0aa230090948800c09b230064
:1039f000a0948800e08c2300b0948800307e2300df
:103a0000c0948800d06f2300d0948800a061230068
:103a1000e0948800b0532300f0948800f045230020
:103a2000009588007038230010958800202b230013
:103a300020958800101e2300309588004011230037
:103a400040958800900423005095880020f82200bb
:103a500060958800e0eb220070958800d0df22009e
:103a600080958800f0d322009095880050c82200ed
:103a7000a0958800d0bc2200b095880080b12200bb
:103a8000c095880070a62200d0958800809b2200f7
:103a9000e0958800c0902200f095880020862200e2
:103aa00000968800c07b220010968800807122005a
:103ab000209688006067220030968800805d220092
:103ac00040968800c053220050968800204a220069
:103ad00060968800b040220070968800603722000f
:103ae00080968800402e2200909688004025220073
:103af000a0968800601c2200b0968800b0132200b7
:103b0000c0968800200b2200d0968800b0022200c8
:103b1000e096880060fa2100f096880040f22100cb
:103b20000097880030ea21001097880050e22100b9
:103b30002097880090da210030978800e0d2210099
:103b40004097880060cb210050978800f0c3210087
:103b500060978800b0bc21007097880080b5210074
:103b60008097880080ae21009097880090a7210060
:103b7000a0978800b0a02100b0978800009a21008b
:103b8000c097880060932100d0978800e08c2100c6
:103b9000e097880080862100f0978800308021001f
:103ba00000988800007a210010988800f0732100a6
:103bb00020988800f06d210030988800006821006e
:103bc000409888004062210050988800805c210065
:103bd00060988800e05621007098880060512100ac
:103be00080988800f04b2100909888009046210032
:103bf000a098880050412100b0988800203c210006
:103c0000c098880010372100d09888001032210019
:103c1000e0988800202d2100f0988800402821009d
:103c2000009988008023210010998800d01e21006f
:103c300020998800301a210030998800a0152100b1
:103c4000409988002011210050998800c00c210063
:103c50006099880070082100709988002004210074
:103c600080998800f0ff200090998800d0fb200008
:103c7000a0998800c0f72000b0998800d0f32000f8
:103c8000c0998800e0ef2000d099880000ec200067
:103c9000e099880030e82000f099880070e4200066
:103ca000009a8800c0e02000109a880020dd2000e3
:103cb000209a880090d92000309a880010d62000e1
:103cc000409a8800a0d22000509a880040cf20005f
:103cd000609a8800e0cb2000709a8800a0c820007d
:103ce000809a880060c52000909a880030c2200029
:103cf000a09a880010bf2000b09a880000bc200065
:103d0000c09a88000000060030b62f00309c880062
:103d100070d42e00409c880060ff2d00509c8800cd
:103d200040362d00609c880070782c00709c8800c4
:103d300040c52b00809c8800201c2b00909c880094
:103d4000807c2a00a09c8800d0e52900b09c8800d7
:103d5000a0572900c09c880060d12800d09c880012
:103d6000b0522800e09c880020db2700f09c8800ef
:103d7000406a2700009d8800b0ff2600109d880043
:103d8000209b2600209d8800303c2600309d880026
:103d9000a0e22500409d8800108e2500509d8800df
:103da000403e2500609d8800f0f22400709d880050
:103db000d0ab2400809d8800b0682400909d8800ce
:103dc00050292400a09d880090ed2300b09d88001c
:103dd00020b52300c09d8800d07f2300d09d88009f
:103de000904d2300e09d8800201e2300f09d880058
:103df00050f12200009e880000c72200109e88001b
:103e0000209f2200209e880070792200309e88002a
:103e1000e0552200409e880060342200509e8800b9
:103e2000b0142200609e8800c0f62100709e8800b9
:103e300090da2100809e8800f0bf2100909e8800cb
:103e4000c0a62100a09e8800108f2100b09e88008f
:103e5000a0782100c09e880080632100d09e880049
:103e6000904f2100e09e8800c03c2100f09e880019
:103e7000f02a2100009f8800301a2100109f88003e
:103e8000500a2100209f880060fb2000309f88009e
:103e900040ed2000409f8800f0df2000509f880008
:103ea00060d32000609f880080c72000709f88003a
:103eb00050bc2000809f8800c0b12000909f8800e7
:103ec000c0a72000a09f8800609e2000b09f8800af
:103ed00080952000c09f8800108d2000d09f880012
:103ee00030852000e09f8800b07d2000f09f880092
:103ef000a076200000a088000070200010a088009c
:103f0000b069200020a08800c063200030a0880095
:103f1000305e200040a08800e058200050a08800bb
:103f2000e053200060a08800304f200070a088007f
:103f3000c04a200080a088009046200090a0880001
:103f400090422000a0a08800e03e2000b0a08800a1
:103f5000503b2000c0a0880000382000d0a088007e
:103f6000e0342000e0a08800e0312000f0a08800cc
:103f7000102f200000a18800702c200010a18800c4
:103f8000f029200020a188009027200030a188007f
:103f90006025200040a188004023200050a1880017
:103fa0005021200060a18800701f200070a18800af
:103fb000b01d200080a18800001c200090a1880076
:103fc000701a2000a0a18800f0182000b0a188007d
:103fd00090172000c0a1880040162000d0a18800c2
:103fe00000152000e0a18800d0132000f0a1880077
:103ff000b012200000a28800a011200010a28800aa
:10400000a010200020a28800b00f200030a288005d
:10401000d00e200040a28800000e200050a2880090
:10402000300d200060a28800800c200070a2880063
:10403000c00b200080a28800200b200090a28800e6
:10404000800a2000a0a28800e0092000b0a2880019
:1040500050092000c0a28800000006005a34ef007a
:10406000a0a82100e0a2880050b02100f0a28800a2
:1040700030b8210000a3880020c0210010a38800d0
:1040800050c8210020a3880090d0210030a38800d0
:1040900000d9210040a3880090e1210050a38800ae
:1040a00050ea210060a3880040f3210070a388003b
:1040b00050fc210080a388008005220090a3880086
:1040c000f00e2200a0a3880080182200b0a3880070
:1040d00030222200c0a38800202c2200d0a3880018
:1040e00040362200e0a3880080402200f0a3880030
:1040f000f04a220000a48800a055220010a48800e5
:104100007060220020a48800806b220030a4880008
:10411000c076220040a488003082220050a488008b
:10412000e08d220060a48800c099220070a488005d
:10413000d0a5220080a4880020b2220090a488008c
:10414000a0be2200a0a4880060cb2200b0a48800fa
:1041500060d82200c0a48800a0e52200d0a4880076
:1041600010f32200e0a48800c0002300f0a488001f
:10417000c00e230000a58800f01c230010a58800b5
:10418000602b230020a58800203a230030a588005a
:104190002049230040a588006058230050a58800ce
:1041a000f067230060a58800c077230070a5880011
:1041b000e087230080a588005098230090a5880000
:1041c00000a92300a0a5880000ba2300b0a588009c
:1041d00050cb2300c0a58800f0dc2300d0a58800c8
:1041e000e0ee2300e0a5880030012400f0a588005f
:1041f000d013240000a68800c026240010a6880042
:10420000003a240020a68800b04d240030a6880083
:10421000b061240040a688000076240050a68800e3
:10422000c08a240060a68800e09f240070a6880051
:1042300050b5240080a6880040cb240090a68800ba
:1042400080e12400a0a6880030f82400b0a68800f1
:10425000400f2500c0a68800c0262500d0a68800f3
:10426000b03e2500e0a6880010572500f0a6880083
:10427000e06f250000a788003089250010a788007e
:10428000e0a2250020a7880010bd250030a78800e7
:10429000c0d7250040a78800e0f2250050a788007d
:1042a000900e260060a78800b02a260070a788001c
:1042b0006047260080a788008064260090a78800b9
:1042c00040822600a0a7880080a02600b0a7880012
:1042d00040bf2600c0a78800a0de2600d0a7880027
:1042e00090fe2600e0a78800101f2700f0a7880096
:1042f0002040270000a88800d061270010a888006f
:104300002084270020a8880010a7270030a8880054
:10431000a0ca270040a88800d0ee270050a8880037
:10432000b013280060a888004039280070a88800d1
:10433000705f280080a888005086280090a8880018
:10434000f0ad2800a0a8880050d62800b0a88800aa
:1043500060ff2800c0a8880030292900d0a8880064
:10436000c0532900e0a88800107f2900f0a8880029
:1043700030ab290000a9880020d8290010a98800a6
:10438000e0052a0020a9880070342a0030a988009e
:10439000e0632a0040a9880020942a0050a98800e0
:1043a00050c52a0060a9880060f72a0070a988001b
:1043b000502a2b0080a98800305e2b0090a988002d
:1043c00000932b00a0a98800d0c82b00b0a98800ba
:1043d00090ff2b00c0a9880050372c00d0a988007e
:1043e00010702c00e0a98800e0a92c00f0a988003a
:1043f000c0e42c0000aa8800a0202d0010aa88008c
:10440000a05d2d0020aa8800c09b2d0030aa880046
:1044100000db2d0040aa8800601b2e0050aa8800f7
:10442000f05c2e0060aa8800b09f2e0070aa880061
:10443000a0e32e0080aa8800d0282f0090aa880030
:10444000406f2f00a0aa880000b72f00b0aa8800f4
:1044500058b5ef00110037004f72ef00f0c7b300fe
:104460004f52e3000d003e004fd2bf000080fb0022
:1044700000004000a145210060807800f124210067
:10448000914078008180fb0081804000a24521009e
:10449000803079004f72ec00f0ff39000000060018
:1044a0005a34ef00b0882000e0a28800708c200011
:1044b000f0a288005090200000a3880040942000c3
:1044c00010a388005098200020a38800709c200032
:1044d00030a38800c0a0200040a3880020a52000b1
:1044e00050a38800a0a9200060a3880050ae20003f
:1044f00070a3880010b3200080a38800f0b72000cc
:1045000090a3880000bd2000a0a3880020c2200046
:10451000b0a3880070c72000c0a38800f0cc2000a2
:10452000d0a3880080d22000e0a3880040d82000db
:10453000f0a3880030de200000a4880040e42000c2
:1045400010a4880080ea200020a48800f0f0200059
:1045500030a4880080f7200040a4880050fe20008e
:1045600050a488004005210060a48800600c210050
:1045700070a48800c013210080a48800401b210083
:1045800090a4880000232100a0a48800002b210013
:10459000b0a4880030332100c0a48800903b2100e3
:1045a000d0a4880030442100e0a48800104d2100f0
:1045b000f0a488003056210000a58800805f21000b
:1045c00010a588002069210020a588000073210023
:1045d00030a58800307d210040a58800908721000b
:1045e00050a588005092210060a58800509d2100b0
:1045f00070a58800a0a8210080a5880030b4210003
:1046000090a5880020c02100a0a5880060cc2100d2
:10461000b0a5880000d92100c0a58800f0e52100e0
:10462000d0a5880040f32100e0a58800e00022002a
:10463000f0a58800f00e220000a68800501d220080
:1046400010a68800202c220020a68800503b2200c3
:1046500030a68800f04a220040a68800005b2200b5
:1046600050a68800806b220060a68800707c220023
:1046700070a68800e08d220080a68800c09f2200de
:1046800090a6880020b22200a0a6880000c52200c3
:10469000b0a6880060d82200c0a6880050ec220096
:1046a000d0a68800c0002300e0a68800d015230013
:1046b000f0a68800602b230000a78800904123000b
:1046c00010a788006058230020a78800d06f23001f
:1046d00030a78800e087230040a78800a0a023001f
:1046e00050a7880000ba230060a7880010d42300d8
:1046f00070a78800e0ee230080a78800700a2400dd
:1047000090a78800c0262400a0a78800d0432400da
:10471000b0a78800b0612400c0a7880050802400a2
:10472000d0a78800e09f2400e0a7880040c02400b4
:10473000f0a7880080e1240000a88800b0032500cd
:1047400010a88800c026250020a88800e04a25007f
:1047500030a88800e06f250040a88800009625005a
:1047600050a8880010bd250060a8880040e52500fd
:1047700070a88800900e260080a88800f0382600d7
:1047800090a8880080642600a0a888005091260088
:10479000b0a8880040bf2600c0a8880080ee260090
:1047a000d0a88800101f2700e0a88800f05027003c
:1047b000f0a888002084270000a98800c0b827003e
:1047c00010a98800d0ee270020a9880060262800c4
:1047d00030a98800705f280040a98800109a28003e
:1047e00050a9880050d6280060a9880030142900fc
:1047f00070a98800c053290080a98800109529005d
:1048000090a9880020d82900a0a98800101d2a009e
:10481000b0a98800e0632a00c0a98800a0ac2a00e3
:10482000d0a9880060f72a00e0a9880020442b0066
:10483000f0a9880000932b0000aa880010e42b0048
:1048400010aa880050372c0020aa8800e08c2c0089
:1048500030aa8800c0e42c0040aa8800003f2d0048
:1048600050aa8800c09b2d0060aa880010fb2d0074
:1048700070aa8800f05c2e0080aa880080c12e00fb
:1048800090aa8800d0282f00a0aa8800f0922f00bc
:10489000b0aa880058b5ef00110037004f72ef0042
:1048a000f0c7b3004f52e3000d003e004fd2bf00ef
:1048b0000080fb0000004000a145210060807800de
:1048c000f1242100914078008180fb00818040002c
:1048d000a2452100803079004f72ec00f0ff3900d2
:1048e000000006005a34ef00002c2000e0a28800ef
:1048f000a02d2000f0a28800502f200000a38800e7
:104900001031200010a38800d032200020a388009e
:10491000b034200030a38800a036200040a38800d7
:10492000a038200050a38800b03a200060a388007f
:10493000e03c200070a38800103f200080a3880086
:104940006041200090a38800d0432000a0a38800ed
:1049500040462000b0a38800d0482000c0a38800b3
:10496000804b2000d0a38800404e2000e0a38800a8
:1049700020512000f0a388002054200000a48800cb
:104980003057200010a48800605a200020a488001e
:10499000b05d200030a488002061200040a4880081
:1049a000b064200050a488006068200060a48800e3
:1049b000306c200070a488003070200080a4880033
:1049c0004074200090a4880090782000a0a4880063
:1049d000f07c2000b0a4880080812000c0a4880062
:1049e00040862000d0a48800308b2000e0a48800fe
:1049f00050902000f0a488009095200000a5880029
:104a0000109b200010a58800c0a0200020a58800d1
:104a1000a0a6200030a58800c0ac200040a58800da
:104a200010b3200050a58800a0b9200060a5880020
:104a300070c0200070a5880070c7200080a5880085
:104a4000c0ce200090a5880050d62000a0a58800e8
:104a500030de2000b0a5880050e62000c0a5880008
:104a6000c0ee2000d0a5880080f72000e0a58800d7
:104a700090002100f0a58800000a210000a688000f
:104a8000c013210010a68800d01d210020a6880098
:104a90005028210030a688003033210040a688002d
:104aa000703e210050a68800104a210060a68800b0
:104ab0003056210070a68800b062210080a68800d0
:104ac000b06f210090a68800307d2100a0a688004c
:104ad000208b2100b0a68800a0992100c0a68800e4
:104ae000a0a82100d0a6880030b82100e0a6880048
:104af00050c82100f0a6880000d9210000a7880036
:104b000050ea210010a7880050fc210020a788004f
:104b1000f00e220030a788003022220040a7880033
:104b20004036220050a78800f04a220060a7880083
:104b30007060220070a78800c076220080a78800dd
:104b4000e08d220090a78800d0a52200a0a78800b1
:104b5000a0be2200b0a7880060d82200c0a78800ad
:104b600010f32200d0a78800c00e2300e0a7880021
:104b7000602b2300f0a788002049230000a88800ac
:104b8000f067230010a88800e087230020a8880091
:104b900000a9230030a8880050cb230040a888003b
:104ba000e0ee230050a88800d013240060a88800fd
:104bb000003a240070a88800b061240080a8880012
:104bc000c08a240090a8880050b52400a0a88800be
:104bd00080e12400b0a88800400f2500c0a888000c
:104be000b03e2500d0a88800e06f2500e0a888002e
:104bf000e0a22500f0a88800c0d7250000a9880001
:104c0000900e260010a988006047260020a9880081
:104c10004082260030a9880040bf260040a98800b5
:104c200090fe260050a988002040270060a9880037
:104c30002084270070a98800a0ca270080a98800c6
:104c4000b013280090a98800705f2800a0a98800f0
:104c5000f0ad2800b0a9880060ff2800c0a9880036
:104c6000c0532900d0a9880030ab2900e0a98800f2
:104c7000e0052a00f0a98800e0632a0000aa880065
:104c800050c52a0010aa8800502a2b0020aa8800ac
:104c900000932b0030aa880090ff2b0040aa8800c8
:104ca00010702c0050aa8800c0e42c0060aa880074
:104cb000a05d2d0070aa880000db2d0080aa88006e
:104cc000f05c2e0090aa8800a0e32e00a0aa880025
:104cd000406f2f00b0aa880058b5ef0011003700d0
:104ce0004f72ef00f0c7b3004f52e3000d003e00db
:104cf0004fd2bf000080fb0000004000a145210012
:104d000060807800f1242100914078008180fb00d0
:104d100081804000a2452100803079004f72ec0074
:104d2000f0ff3900000006005a34ef00300e20007a
:104d3000e0a28800d00e2000f0a28800800f2000a2
:104d400000a388003010200010a38800f01020007d
:104d500020a38800c011200030a3880090122000fa
:104d600040a388007013200050a388005014200036
:104d700060a388004015200070a388004016200022
:104d800080a388004017200090a3880050182000be
:104d9000a0a3880070192000b0a38800a01a2000ea
:104da000c0a38800d01b2000d0a38800201d2000b5
:104db000e0a38800701e2000f0a38800d01f200010
:104dc00000a488005021200010a48800d0222000d8
:104dd00020a488007024200030a488002026200011
:104de00040a48800e027200050a48800b0292000bb
:104df00060a48800a02b200070a48800a02d2000b3
:104e000080a48800c02f200090a48800f0312000ea
:104e1000a0a4880040342000b0a48800a036200060
:104e2000c0a4880020392000d0a48800c03b200006
:104e3000e0a48800803e2000f0a4880060412000ab
:104e400000a588006044200010a58800904720003d
:104e500020a58800d04a200030a58800404e2000c0
:104e600040a58800e051200050a58800a0552000f2
:104e700060a588009059200070a58800b05d2000d2
:104e800080a588000062200090a588008066200030
:104e9000a0a58800406b2000b0a5880030702000dd
:104ea000c0a5880050752000d0a58800c07a2000d9
:104eb000e0a5880060802000f0a5880040862000e2
:104ec00000a68800708c200010a68800f0922000b8
:104ed00020a68800b099200030a68800c0a020003d
:104ee00040a6880020a8200050a68800e0af20003f
:104ef00060a68800f0b7200070a6880070c020006f
:104f000080a6880040c9200090a6880080d220009a
:104f1000a0a6880030dc2000b0a6880050e6200063
:104f2000c0a68800f0f02000d0a6880000fc200079
:104f3000e0a68800a0072100f0a68800c013210089
:104f400000a788007020210010a78800b02d210044
:104f500020a78800903b210030a78800104a21003c
:104f600040a788004059210050a7880020692100ef
:104f700060a78800c079210070a78800208b2100dd
:104f800080a78800509d210090a7880050b0210084
:104f9000a0a7880030c42100b0a7880000d9210054
:104fa000c0a78800c0ee2100d0a78800800522009d
:104fb000e0a78800501d2200f0a78800403622009c
:104fc00000a888004050220010a88800806b2200b2
:104fd00020a888000088220030a88800d0a52200e0
:104fe00040a8880000c5220050a88800a0e5220043
:104ff00060a88800b007230070a88800602b2300f9
:1050000080a88800c050230090a88800c0772300a3
:10501000a0a88800a0a02300b0a8880050cb23003f
:10502000c0a8880000f82300d0a88800c02624006b
:10503000e0a88800a0572400f0a88800c08a2400b7
:1050400000a9880040c0240010a9880030f824007e
:1050500020a98800b032250030a98800e06f250023
:1050600040a98800f0af250050a98800e0f2250093
:1050700060a98800f038260070a9880040822600c8
:1050800080a98800e0ce260090a98800101f270084
:10509000a0a98800e0722700b0a98800a0ca270054
:1050a000c0a9880060262800d0a988005086280062
:1050b000e0a98800c0ea2800f0a98800c0532900b0
:1050c00000aa880090c1290010aa880070342a0024
:1050d00020aa8800a0ac2a0030aa8800502a2b0001
:1050e00040aa8800d0ad2b0050aa880050372c0071
:1050f00060aa880030c72c0070aa8800a05d2d002f
:1051000080aa880010fb2d0090aa8800b09f2e0076
:10511000a0aa8800e04b2f00b0aa880058b5ef0085
:10512000110037004f72ef00f0c7b3004f52e30099
:105130000d003e004fd2bf000080fb000000400089
:10514000a145210060807800f12421009140780081
:105150008180fb0081804000a245210080307900e1
:105160004f72ec00f0ff3900000006005a34ef00e7
:1051700090042000e0a28800d0042000f0a2880063
:105180001005200000a388006005200010a38800ff
:10519000b005200020a388000006200030a388006e
:1051a0005006200040a38800b006200050a38800cd
:1051b0000007200060a388007007200070a388000b
:1051c000d007200080a388004008200090a388001a
:1051d000c0082000a0a3880030092000b0a38800e8
:1051e000b0092000c0a38800400a2000d0a3880096
:1051f000d00a2000e0a38800700b2000f0a38800f4
:10520000100c200000a48800c00c200010a488000e
:10521000700d200020a48800300e200030a48800eb
:10522000f00e200040a48800d00f200050a4880079
:10523000b010200060a488009011200070a48800a5
:105240009012200080a488009013200090a4880071
:10525000b0142000a0a48800d0152000b0a48800bd
:1052600010172000c0a4880050182000d0a4880087
:10527000b0192000e0a48800101b2000f0a48800d2
:10528000901c200000a58800301e200010a588007a
:10529000d01f200020a58800a021200030a5880074
:1052a0008023200040a588007025200050a588009c
:1052b0008027200060a58800b029200070a5880004
:1052c000002c200080a58800702e200090a588006a
:1052d00010312000a0a58800c0332000b0a58800b0
:1052e000a0362000c0a58800a0392000d0a58800e5
:1052f000e03c2000e0a5880040402000f0a58800a8
:10530000d043200000a688009047200010a6880007
:10531000804b200020a68800b04f200030a68800d7
:105320002054200040a68800c058200050a68800c5
:10533000b05d200060a68800e062200070a68800b2
:105340006068200080a68800306e200090a688004b
:1053500040742000a0a68800c07a2000b0a6880073
:1053600080812000c0a68800b0882000d0a68800d8
:1053700050902000e0a6880050982000f0a68800f9
:10538000c0a0200000a78800a0a9200010a78800c6
:1053900010b3200020a7880000bd200030a788009f
:1053a00070c7200040a7880080d2200050a7880046
:1053b00030de200060a7880080ea200070a7880007
:1053c00080f7200080a788004005210090a7880072
:1053d000c0132100a0a7880000232100b0a78800e7
:1053e00030332100c0a7880030442100d0a78800b6
:1053f00030562100e0a7880020692100f0a788002e
:10540000307d210000a888005092210010a888005b
:10541000a0a8210020a8880020c0210030a8880072
:1054200000d9210040a8880040f3210050a888003e
:10543000f00e220060a88800202c220070a88800ae
:10544000f04a220080a88800806b220090a8880083
:10545000e08d2200a0a8880020b22200b0a8880019
:1054600060d82200c0a88800c0002300d0a888000f
:10547000602b2300e0a8880060582300f0a8880073
:10548000e087230000a9880000ba230010a9880043
:10549000e0ee230020a98800c026240030a988005f
:1054a000b061240040a98800e09f240050a9880032
:1054b00080e1240060a98800c026250070a988002a
:1054c000e06f250080a9880010bd250090a9880004
:1054d000900e2600a0a9880080642600b0a988004c
:1054e00040bf2600c0a98800101f2700d0a988004f
:1054f00020842700e0a98800d0ee2700f0a98800ca
:10550000705f280000aa880050d6280010aa8800e2
:10551000c053290020aa880020d8290030aa88007a
:10552000e0632a0040aa880060f72a0050aa880099
:1055300000932b0060aa880050372c0070aa8800c6
:10554000c0e42c0080aa8800c09b2d0090aa88008f
:10555000f05c2e00a0aa8800d0282f00b0aa8800f6
:1055600058b5ef00110037004f72ef00f0c7b300dd
:105570004f52e3000d003e004fd2bf000080fb0001
:1055800000004000a145210060807800f124210046
:10559000914078008180fb0081804000a24521007d
:1055a000803079004f72ec00f0ff390000000600f7
:0455b000ffff3700c2
:020000040000fa
:1055b400d41100000800000080000000dc1100008d
:1055c4001e00000080000000fa11000044000000ea
:1055d400800000003e1200001c000000800000005b
:1055e4005a12000000030000800000005a15000059
:0c55f4000001000080000000000000002a
:00000001FF
